 libOpenVG

 Timestamp is 4be8c51d (Tue May 11 11:46:53 2010)

 Preferred load address is 10000000

 Start         Length     Name                   Class
 0001:00000000 00000004H .CRT$XCA                CODE
 0001:00000004 00000004H .CRT$XCZ                CODE
 0001:00000008 00000004H .CRT$XIA                CODE
 0001:0000000c 00000004H .CRT$XIZ                CODE
 0001:00000010 00000004H .CRT$XPA                CODE
 0001:00000014 00000004H .CRT$XPZ                CODE
 0001:00000018 00000004H .CRT$XTA                CODE
 0001:0000001c 00000004H .CRT$XTZ                CODE
 0001:00000020 0001c778H .rdata                  CODE
 0001:0001c798 00000026H .rdata$debug            CODE
 0001:0001c7c0 0004bbf8H .text                   CODE
 0001:000683b8 00000024H .xdata                  CODE
 0001:000683dc 0000003cH .idata$2                CODE
 0001:00068418 00000014H .idata$3                CODE
 0001:0006842c 00000158H .idata$4                CODE
 0001:00068584 000000c4H .idata$6                CODE
 0001:00068650 00000838H .edata                  CODE
 0002:00000000 00000158H .idata$5                DATA
 0002:00000158 0000000cH .data                   DATA
 0002:00000164 00000014H .bss                    DATA
 0003:00000000 00001020H .pdata                  DATA

  Address         Publics by Value              Rva+Base       Lib:Object

 0000:00000000       ___safe_se_handler_table   00000000     <absolute>
 0000:00000000       ___safe_se_handler_count   00000000     <absolute>
 0001:00000000       __xc_a                     10001000     corelib0:crt0init.obj
 0001:00000004       __xc_z                     10001004     corelib0:crt0init.obj
 0001:00000008       __xi_a                     10001008     corelib0:crt0init.obj
 0001:0000000c       __xi_z                     1000100c     corelib0:crt0init.obj
 0001:00000010       __xp_a                     10001010     corelib0:crt0init.obj
 0001:00000014       __xp_z                     10001014     corelib0:crt0init.obj
 0001:00000018       __xt_a                     10001018     corelib0:crt0init.obj
 0001:0000001c       __xt_z                     1000101c     corelib0:crt0init.obj
 0001:00004398       ??_C@_03GCKCNDHP@1?41?$AA@ 10005398     get.obj
 0001:0000439c       ??_C@_0BA@HGHHDPMC@PowerVR?5SGX?5540?$AA@ 1000539c     get.obj
 0001:000043ac       ??_C@_0BJ@FGEHHHOH@Imagination?5Technologies?$AA@ 100053ac     get.obj
 0001:00004a88       ??_C@_0BK@MJMMJBHE@vgCreateEGLImageTargetKHR?$AA@ 10005a88     get.obj
 0001:00009148       ??_C@_0BP@CGBHEOOJ@DefaultPregenPDSVertBufferSize?$AA@ 1000a148     util.obj
 0001:00009168       ??_C@_0BJ@OAODBGJG@DefaultSpecObjBufferSize?$AA@ 1000a168     util.obj
 0001:00009184       ??_C@_0BJ@FDELEOJK@DefaultPDSVertBufferSize?$AA@ 1000a184     util.obj
 0001:000091a0       ??_C@_0BJ@GGBNLCGB@DefaultPDSFragBufferSize?$AA@ 1000a1a0     util.obj
 0001:000091bc       ??_C@_0BF@GMGALNEL@DefaultVDMBufferSize?$AA@ 1000a1bc     util.obj
 0001:000091d4       ??_C@_0L@CDGAGNFA@KickTAMode?$AA@ 1000a1d4     util.obj
 0001:000091e0       ??_C@_0BA@FMCJLEC@KickTAThreshold?$AA@ 1000a1e0     util.obj
 0001:0001e4b0       OVGCreateGC                1001f4b0 f   eglglue.obj
 0001:0001e568       OVGContext_dealloc         1001f568 f   eglglue.obj
 0001:0001e680       OVGDestroyGC               1001f680 f   eglglue.obj
 0001:0001e6a0       OVGMakeCurrentGC           1001f6a0 f   eglglue.obj
 0001:0001e930       OVGMakeUnCurrentGC         1001f930 f   eglglue.obj
 0001:0001eb68       OVGUnWrapImage             1001fb68 f   eglglue.obj
 0001:0001eb94       OVGWrapImageAsRenderSurface 1001fb94 f   eglglue.obj
 0001:0001ef24       OVGGetRenderSurface        1001ff24 f   eglglue.obj
 0001:0001ef2c       OVGGetDrawableParams       1001ff2c f   eglglue.obj
 0001:0001ef34       OVGFlushBuffersGC          1001ff34 f   eglglue.obj
 0001:0001f144       OVGComputeQuadBezierTangent 10020144 f   splines.obj
 0001:0001f3b4       OVGComputeCubicBezierTangent 100203b4 f   splines.obj
 0001:0001f914       OVGSuggestCubicBezierTessMetric 10020914 f   splines.obj
 0001:0001fcc0       OVGCalculateQuadBezierTangents 10020cc0 f   splines.obj
 0001:0001ff1c       OVGCalculateCubicBezierTangents 10020f1c f   splines.obj
 0001:000201d8       OVGPointAlongCatmulRomSpline 100211d8 f   splines.obj
 0001:00020834       OVGCalculateExtraControlPoint 10021834 f   splines.obj
 0001:00020b70       OVGComputeCubicBezier      10021b70 f   splines.obj
 0001:00020dc4       OVGComputeCubicBezierLength 10021dc4 f   splines.obj
 0001:00020e98       OVGComputeQuadBezier       10021e98 f   splines.obj
 0001:00020ff4       OVGComputeQuadBezierLength 10021ff4 f   splines.obj
 0001:000211a4       OVGFindUnitCircleCentre    100221a4 f   ellipse.obj
 0001:000214cc       OVGCircumferenceOfEllipse  100224cc f   ellipse.obj
 0001:00021568       OVGFindEllipse             10022568 f   ellipse.obj
 0001:00021cb0       OVGFindEllipseTangents     10022cb0 f   ellipse.obj
 0001:00022418       OVGSuggestEllipticalArcTessMetric 10023418 f   ellipse.obj
 0001:000226b4       OVGComputeEllipticalArcLength 100236b4 f   ellipse.obj
 0001:00022c40       OVGFloorLog2               10023c40 f   maths.obj
 0001:00022c60       OVGClampf                  10023c60 f   maths.obj
 0001:00022cc4       OVGComputeBoundingBoxUnion 10023cc4 f   maths.obj
 0001:00022d3c       OVGDoRectsOverlap          10023d3c f   maths.obj
 0001:00022d9c       OVGLoadIdentity            10023d9c f   maths.obj
 0001:00022dc8       OVGMatrixMultiply          10023dc8 f   maths.obj
 0001:000232dc       OVGMatrixInvert            100242dc f   maths.obj
 0001:000237dc       OVGCalculateDeterminant2x2 100247dc f   maths.obj
 0001:0002383c       OVGTransformPoint          1002483c f   maths.obj
 0001:0002535c       OVGTessellateFillPath      1002635c f   tessellate.obj
 0001:00026f60       OVGTessellateStrokeJoins   10027f60 f   tessellate.obj
 0001:00027e2c       OVGTessellateStrokeCaps    10028e2c f   tessellate.obj
 0001:00028e94       OVGTessellateStrokePath    10029e94 f   tessellate.obj
 0001:0002b7cc       OVGTessellateDashedStroke  1002c7cc f   tessellate.obj
 0001:0002c718       vgGetString                1002d718 f   get.obj
 0001:0002c7ac       vgGetf                     1002d7ac f   get.obj
 0001:0002cc8c       vgGeti                     1002dc8c f   get.obj
 0001:0002d098       vgGetVectorSize            1002e098 f   get.obj
 0001:0002d268       vgGetfv                    1002e268 f   get.obj
 0001:0002d63c       vgGetiv                    1002e63c f   get.obj
 0001:0002d9fc       vgGetParameterf            1002e9fc f   get.obj
 0001:0002dda0       vgGetParameteri            1002eda0 f   get.obj
 0001:0002e088       vgGetParameterVectorSize   1002f088 f   get.obj
 0001:0002e1e8       vgGetParameterfv           1002f1e8 f   get.obj
 0001:0002e4cc       vgGetParameteriv           1002f4cc f   get.obj
 0001:0002e7d8       vgGetError                 1002f7d8 f   get.obj
 0001:0002e7fc       vgHardwareQuery            1002f7fc f   get.obj
 0001:0002e8fc       OVGSetError                1002f8fc f   set.obj
 0001:0002e90c       vgSeti                     1002f90c f   set.obj
 0001:0002ecec       vgSetf                     1002fcec f   set.obj
 0001:0002f174       vgSetfv                    10030174 f   set.obj
 0001:0002f930       vgSetiv                    10030930 f   set.obj
 0001:00030038       vgSetParameterf            10031038 f   set.obj
 0001:00030214       vgSetParameteri            10031214 f   set.obj
 0001:000303cc       vgSetParameterfv           100313cc f   set.obj
 0001:00030810       vgSetParameteriv           10031810 f   set.obj
 0001:00030c74       vgFlush                    10031c74 f   set.obj
 0001:00030c78       vgFinish                   10031c78 f   set.obj
 0001:00030ef4       OVGSetupVertexShaderForClear 10031ef4 f   clear.obj
 0001:00031398       OVGSendClear               10032398 f   clear.obj
 0001:000318c4       vgClear                    100328c4 f   clear.obj
 0001:00031a48       OVGRemovePath              10032a48 f   path.obj
 0001:00031b9c       OVGPath_release            10032b9c f   path.obj
 0001:00031bbc       OVGPath_retain             10032bbc f   path.obj
 0001:00031bcc       OVGPath_handle             10032bcc f   path.obj
 0001:00031bd4       OVGPath_setHandle          10032bd4 f   path.obj
 0001:00031bdc       OVGPath_dealloc            10032bdc f   path.obj
 0001:00031be8       vgAppendPathData           10032be8 f   path.obj
 0001:00031e00       vgClearPath                10032e00 f   path.obj
 0001:00031ec0       vgDestroyPath              10032ec0 f   path.obj
 0001:00031f64       vgRemovePathCapabilities   10032f64 f   path.obj
 0001:00032008       vgGetPathCapabilities      10033008 f   path.obj
 0001:000320b0       vgAppendPath               100330b0 f   path.obj
 0001:000321c8       vgModifyPathCoords         100331c8 f   path.obj
 0001:000324dc       vgDrawPath                 100334dc f   path.obj
 0001:000325c4       vgTransformPath            100335c4 f   path.obj
 0001:0003394c       vgInterpolatePath          1003494c f   path.obj
 0001:00033e4c       vgPathLength               10034e4c f   path.obj
 0001:00034840       vgPathBounds               10035840 f   path.obj
 0001:00034c08       vgPathTransformedBounds    10035c08 f   path.obj
 0001:00034fe8       vgPointAlongPath           10035fe8 f   path.obj
 0001:000354a4       OVGPath_setDirty           100364a4 f   path.obj
 0001:000354b4       vgCreatePath               100364b4 f   path.obj
 0001:0003581c       OVGInitialiseFrameResManagers 1003681c f   meminstance.obj
 0001:000358fc       OVGDestroyFrameResManagers 100368fc f   meminstance.obj
 0001:00035928       OVGFreeRedundantMem        10036928 f   meminstance.obj
 0001:000359ac       OVGFreeMemInstance         100369ac f   meminstance.obj
 0001:00035a38       OVGFreeRedundantMemList    10036a38 f   meminstance.obj
 0001:00035b1c       OVGAllocGeneralHeapDeviceMem 10036b1c f   meminstance.obj
 0001:00035da8       OVGCleanupRedundantMemInstances 10036da8 f   meminstance.obj
 0001:00035eb4       OVGCreateMemInstance       10036eb4 f   meminstance.obj
 0001:00035f34       OVGGhostMemInstance        10036f34 f   meminstance.obj
 0001:000360b8       OVGCreatePrimitive         100370b8 f   primitive.obj
 0001:000361b4       OVGAttachIndexBufferBatch  100371b4 f   primitive.obj
 0001:000362c8       OVGDestroyPrimitive        100372c8 f   primitive.obj
 0001:00036394       OVGGetCodeBlockHashValue   10037394 f   statehash.obj
 0001:000363f8       OVGHashCodeBlock           100373f8 f   statehash.obj
 0001:00036450       OVGMatchWithHashedCodeBlock 10037450 f   statehash.obj
 0001:000364f8       OVGFreeAllHashedCodeBlocks 100374f8 f   statehash.obj
 0001:00036550       OVGSubmitObject            10037550 f   statehash.obj
 0001:00036680       OVGRetrieveObjectWithType  10037680 f   statehash.obj
 0001:000366c4       OVGRetrieveObject          100376c4 f   statehash.obj
 0001:00036700       OVGInvalidateHandle        10037700 f   statehash.obj
 0001:00036784       OVGCleanObjectPool         10037784 f   statehash.obj
 0001:00036c10       OVGPaint_pixelShaderiseForTAG 10037c10 f   paint.obj
 0001:00036e30       OVGPaint_setNeedsTokenising 10037e30 f   paint.obj
 0001:00036e3c       OVGCreatePaintObject       10037e3c f   paint.obj
 0001:00036ef8       OVGRemovePaint             10037ef8 f   paint.obj
 0001:00036fa4       OVGCreateDefaultColourRamp 10037fa4 f   paint.obj
 0001:000372e0       OVGCreateColourRamp        100382e0 f   paint.obj
 0001:00037fc0       OVGSetLinearGradientUVTransform 10038fc0 f   paint.obj
 0001:00038328       OVGSetPatternUVTransform   10039328 f   paint.obj
 0001:00038404       OVGRemoveCurrentPaint      10039404 f   paint.obj
 0001:0003848c       vgCreatePaint              1003948c f   paint.obj
 0001:0003851c       vgGetPaint                 1003951c f   paint.obj
 0001:000385c4       vgSetColor                 100395c4 f   paint.obj
 0001:0003865c       vgGetColor                 1003965c f   paint.obj
 0001:000386fc       vgPaintPattern             100396fc f   paint.obj
 0001:000387fc       OVGPaint_tokenise          100397fc f   paint.obj
 0001:00038f90       OVGPaint_release           10039f90 f   paint.obj
 0001:00038fb0       OVGPaintResourceUpdate     10039fb0 f   paint.obj
 0001:0003906c       vgDestroyPaint             1003a06c f   paint.obj
 0001:00039118       vgSetPaint                 1003a118 f   paint.obj
 0001:000392bc       OVGWaitForTA               1003a2bc f   sgxif.obj
 0001:00039300       OVGWaitForRender           1003a300 f   sgxif.obj
 0001:0003978c       OVGScheduleTA              1003a78c f   sgxif.obj
 0001:00039bb0       OVGChangeDrawableParams    1003abb0 f   sgxif.obj
 0001:00039c18       OVGKickSmallTA             1003ac18 f   sgxif.obj
 0001:00039c98       OVGKickLimit_ScheduleTA    1003ac98 f   sgxif.obj
 0001:00039cc8       OVGPrepareToDraw           1003acc8 f   sgxif.obj
 0001:00039ed0       OVGInternalFlushBuffers    1003aed0 f   sgxif.obj
 0001:00039f90       OVGSetupUSSEFragmentCodeForAccumulate 1003af90 f   useprog.obj
 0001:0003a034       OVGSetupUSSEFragmentCodeForTQBlit 1003b034 f   useprog.obj
 0001:0003a164       OVGCreateDummyPixelPDSProgram 1003b164 f   useprog.obj
 0001:0003a288       OVGSetupNOPPixelShader     1003b288 f   useprog.obj
 0001:0003a35c       OVGEncodeDmaBurst          1003b35c f   util.obj
 0001:0003a408       OVGGetApplicationHints     1003b408 f   util.obj
 0001:0003a550       OVGColourConvertToHWFormat 1003b550 f   util.obj
 0001:0003a7a0       OVGLoadUSECodeFromHeader   1003b7a0 f   util.obj
 0001:0003a84c       OVGFloatPaintColourToDword 1003b84c f   util.obj
 0001:0003a9b4       OVGOpenVGImageFormatToPixelFormat 1003b9b4 f   util.obj
 0001:0003aafc       OVGOpenVGImageFormatToSGXTextureFormat 1003bafc f   util.obj
 0001:0003ac54       OVGIsSwizzleRequired       1003bc54 f   util.obj
 0001:0003ad30       OVGFormatIsNonLinear       1003bd30 f   util.obj
 0001:0003ad80       OVGFormatIsNonPre          1003bd80 f   util.obj
 0001:0003add0       OVGFormatIsOpaque          1003bdd0 f   util.obj
 0001:0003ae4c       OVGIsPixelScissored        1003be4c f   util.obj
 0001:0003aed4       OVGBuildExtensionString    1003bed4 f   util.obj
 0001:0003aeec       OVGDestroyExtensionString  1003beec f   util.obj
 0001:0003af0c       OVGInputFloatToInt         1003bf0c f   util.obj
 0001:0003afc4       OVGFloatToParam            1003bfc4 f   util.obj
 0001:0003aff8       OVGParamToFloat            1003bff8 f   util.obj
 0001:0003b03c       OVGIntToParam              1003c03c f   util.obj
 0001:0003b084       OVGSetupPixelTaskSizeState 1003c084 f   state.obj
 0001:0003b28c       OVGSetupVertexTaskSizeState 1003c28c f   state.obj
 0001:0003b3d0       OVGIsDestinationRequiredForBlend 1003c3d0 f   state.obj
 0001:0003b4f4       OVGValidateSWStateAndConfigureHWState 1003c4f4 f   state.obj
 0001:0003b770       OVGContext_bitsetCurrentDrawMode 1003c770 f   state.obj
 0001:0003b780       OVGContext_bitunsetCurrentDrawMode 1003c780 f   state.obj
 0001:0003b790       OVGContext_setCurrentDrawMode 1003c790 f   state.obj
 0001:0003b7a4       OVGContext_release         1003c7a4 f   state.obj
 0001:0003b7bc       OVGTokeniseStateForShaders 1003c7bc f   state.obj
 0001:0003bdac       OVGSetupBGObject           1003cdac f   specobj.obj
 0001:0003c018       OVGSetupPixelEventProgram  1003d018 f   specobj.obj
 0001:0003c6d8       OVGSendAccumulateObject    1003d6d8 f   specobj.obj
 0001:0003cbf0       OVGGetPathVertex           1003dbf0 f   pathutils.obj
 0001:0003cc78       OVGSizeofDataType          1003dc78 f   pathutils.obj
 0001:0003ccb4       OVGSegmentRequiredBlockCapacity 1003dcb4 f   pathutils.obj
 0001:0003cd34       OVGCheckConvexity          1003dd34 f   pathutils.obj
 0001:0003cd7c       OVGRecordCurrentStrokeParams 1003dd7c f   pathutils.obj
 0001:0003ce10       OVGAreStrokeParamsDirty    1003de10 f   pathutils.obj
 0001:0003cfa0       OVGSetPathDirty            1003dfa0 f   pathutils.obj
 0001:0003cfb0       OVGGenerateIterativeClipIndices 1003dfb0 f   pathutils.obj
 0001:0003d138       OVGFreeSegmentBlock        1003e138 f   pathutils.obj
 0001:0003d15c       OVGCopyPathSegments        1003e15c f   pathutils.obj
 0001:0003d1e0       OVGCopyAndPromotePathSegments 1003e1e0 f   pathutils.obj
 0001:0003da60       OVGCalculateSegmentLength  1003ea60 f   pathutils.obj
 0001:0003db88       OVGPointAlongSegment       1003eb88 f   pathutils.obj
 0001:0003e614       OVGProcessSegment          1003f614 f   pathutils.obj
 0001:0003ecc4       OVGClassifyPolygon2        1003fcc4 f   convexitytest.obj
 0001:0003fb70       OVGSetDefaultHWState       10040b70 f   hwstate.obj
 0001:0003fb90       OVGSendVertexStateUpdate   10040b90 f   hwstate.obj
 0001:0003fbf0       OVGSendIndexStateUpdate    10040bf0 f   hwstate.obj
 0001:000411ec       _SetUpTextureFilteringBits 100421ec f   pixelshader.obj
 0001:00041250       _SetUpMipMappingBits       10042250 f   pixelshader.obj
 0001:00041e9c       OVGGeneratePixelShader     10042e9c f   pixelshader.obj
 0001:00043288       OVGSetUpBoundingRectVertexBuffer 10044288 f   vertexshader.obj
 0001:00043cac       OVGGenerateVertexShader    10044cac f   vertexshader.obj
 0001:00043e6c       OVGSetupFirstPass          10044e6c f   hwscene.obj
 0001:00043f44       OVGDrawPrimitive           10044f44 f   hwscene.obj
 0001:000441a0       OVGSetPixel                100451a0 f   hwscene.obj
 0001:00044204       OVGPerformOptionalPaintPass 10045204 f   hwscene.obj
 0001:00044380       OVGStrokePath              10045380 f   hwscene.obj
 0001:000445d8       OVGFillPath                100455d8 f   hwscene.obj
 0001:00044674       OVGDrawImage               10045674 f   hwscene.obj
 0001:000450a4       _FromOVGRectToEGLRect      100460a4 f   scissor.obj
 0001:00045188       OVGSendScissorRects        10046188 f   scissor.obj
 0001:0004526c       OVGSendFullScreenEnable    1004626c f   scissor.obj
 0001:00045278       OVGSendRectToStencil       10046278 f   scissor.obj
 0001:0004550c       OVGSendScissorRectsToStencil 1004650c f   scissor.obj
 0001:000455bc       OVGGetMaxScale             100465bc f   matrix.obj
 0001:000456ec       OVGLoadCurrentActiveMatrix 100466ec f   matrix.obj
 0001:00045794       OVGValidateInversePaintMatrix 10046794 f   matrix.obj
 0001:00045804       vgLoadIdentity             10046804 f   matrix.obj
 0001:00045834       vgLoadMatrix               10046834 f   matrix.obj
 0001:000458f4       vgGetMatrix                100468f4 f   matrix.obj
 0001:000459a8       vgMultMatrix               100469a8 f   matrix.obj
 0001:00045a80       vgTranslate                10046a80 f   matrix.obj
 0001:00045af0       vgScale                    10046af0 f   matrix.obj
 0001:00045b60       vgShear                    10046b60 f   matrix.obj
 0001:00045bd0       vgRotate                   10046bd0 f   matrix.obj
 0001:00045d00       OVGPrepareTransferAttributesFromImage 10046d00 f   image.obj
 0001:00045e54       OVGPrepareTransferAttributesFromMemory 10046e54 f   image.obj
 0001:00045f48       OVGPrepareTransferAttributesFromSurface 10046f48 f   image.obj
 0001:00046090       OVGImageCreateSubRegionList 10047090 f   image.obj
 0001:000460c0       OVGImageRetainSubRegionList 100470c0 f   image.obj
 0001:0004611c       OVGImageInvalidateSubRegionList 1004711c f   image.obj
 0001:0004618c       OVGImageReleaseSubRegion   1004718c f   image.obj
 0001:000461f4       OVGImageUpdateSubRegion    100471f4 f   image.obj
 0001:00046348       OVGComputeBlitRegion       10047348 f   image.obj
 0001:00046634       OVGImageRelease            10047634 f   image.obj
 0001:00046654       OVGImageRetain             10047654 f   image.obj
 0001:00046664       OVGImageGetHandle          10047664 f   image.obj
 0001:0004666c       OVGImageSetHandle          1004766c f   image.obj
 0001:00046674       OVGGetImageFormatBytesPerPixel 10047674 f   image.obj
 0001:00046808       OVGRemoveImage             10047808 f   image.obj
 0001:00046908       OVGAlignRectangleWithRenderTarget 10047908 f   image.obj
 0001:00046994       OVGAlignRectangleWithRectangle 10047994 f   image.obj
 0001:000469c8       OVGIntersectRectangleWithRectangle 100479c8 f   image.obj
 0001:00046ab0       OVGIntersectionRect        10047ab0 f   image.obj
 0001:00046b54       vgDestroyImage             10047b54 f   image.obj
 0001:00046bf8       vgClearImage               10047bf8 f   image.obj
 0001:000470c8       vgDrawImage                100480c8 f   image.obj
 0001:00047170       vgGetParent                10048170 f   image.obj
 0001:0004724c       OVGSetPixels               1004824c f   image.obj
 0001:0004744c       vgSetPixels                1004844c f   image.obj
 0001:00047544       vgCopyPixels               10048544 f   image.obj
 0001:00047954       OVGSWBlit                  10048954 f   image.obj
 0001:0004c528       OVGImageGetSubRegion       1004d528 f   image.obj
 0001:0004c6a0       OVGImageDealloc            1004d6a0 f   image.obj
 0001:0004c6ac       OVGCreateImage             1004d6ac f   image.obj
 0001:0004c8dc       vgCreateImage              1004d8dc f   image.obj
 0001:0004ca5c       OVGImageSubData            1004da5c f   image.obj
 0001:0004cc70       vgImageSubData             1004dc70 f   image.obj
 0001:0004cd2c       vgGetImageSubData          1004dd2c f   image.obj
 0001:0004cf3c       vgChildImage               1004df3c f   image.obj
 0001:0004d20c       vgCopyImage                1004e20c f   image.obj
 0001:0004d484       vgWritePixels              1004e484 f   image.obj
 0001:0004d60c       vgGetPixels                1004e60c f   image.obj
 0001:0004d8b0       vgReadPixels               1004e8b0 f   image.obj
 0001:0004db18       OVGGetFormatDescriptor     1004eb18 f   pixelformat.obj
 0001:0004de2c       OVGCheckForValidFBFormat   1004ee2c f   pixelformat.obj
 0001:0004de5c       OVGGetFBFormatDescriptor   1004ee5c f   pixelformat.obj
 0001:0004dfe0       OVGPickPreferedVGImageFormat 1004efe0 f   pixelformat.obj
 0001:0004e12c       SetTwiddledAddrParams      1004f12c f   pixelformat.obj
 0001:0004e180       OVGReadPixelData           1004f180 f   pixelformat.obj
 0001:0004e2c4       OVGWritePixelData          1004f2c4 f   pixelformat.obj
 0001:0004e414       OVGColourConversion        1004f414 f   pixelformat.obj
 0001:0004ec58       _PixelColourConversionScaleBias 1004fc58 f   pixelformat.obj
 0001:0004ee0c       OVGStretchBlitSW           1004fe0c f   pixelformat.obj
 0001:0004f34c       OVGGetTextureLinearAddress 1005034c f   texture.obj
 0001:0004f450       OVGGetTextureDeviceAddress 10050450 f   texture.obj
 0001:0004f510       OVGReferenceTextureInCurrentFrame 10050510 f   texture.obj
 0001:0004f558       OVGCreateTexture           10050558 f   texture.obj
 0001:0004f808       OVGCreateTextureFromEGLImage 10050808 f   texture.obj
 0001:0004f8fc       OVGFreeTexture             100508fc f   texture.obj
 0001:0004f948       OVGInitialiseAlphaMask     10050948 f   mask.obj
 0001:0004f9a0       OVGDestroyAlphaMask        100509a0 f   mask.obj
 0001:00050608       OVGSetupPixelShaderForRenderToMask 10051608 f   mask.obj
 0001:000512d8       OVGRenderMaskBuffer        100522d8 f   mask.obj
 0001:00051500       vgMask                     10052500 f   mask.obj
 0001:000517f8       OVGRemoveMaskLayer         100527f8 f   mask.obj
 0001:0005181c       vgRenderToMask             1005281c f   mask.obj
 0001:00051c50       vgCreateMaskLayer          10052c50 f   mask.obj
 0001:00051d84       vgDestroyMaskLayer         10052d84 f   mask.obj
 0001:00051e44       vgFillMaskLayer            10052e44 f   mask.obj
 0001:00052024       vgCopyMask                 10053024 f   mask.obj
 0001:00052764       DynamicTessellateBezier    10053764 f   subdivide.obj
 0001:00055230       DynamicStrokeBezier        10056230 f   subdivide.obj
 0001:000593ac       vgColorMatrix              1005a3ac f   imagefilter.obj
 0001:000597c8       vgConvolve                 1005a7c8 f   imagefilter.obj
 0001:00059fc8       vgSeparableConvolve        1005afc8 f   imagefilter.obj
 0001:0005f9f8       vgGaussianBlur             100609f8 f   imagefilter.obj
 0001:00060174       vgLookup                   10061174 f   imagefilter.obj
 0001:000607e4       vgLookupSingle             100617e4 f   imagefilter.obj
 0001:00061b14       OVGGenerateRadialGeometry  10062b14 f   radialgradient.obj
 0001:00061f0c       OVGRemoveRadialGradientData 10062f0c f   radialgradient.obj
 0001:00062610       OVGGenerateStencilPassShader 10063610 f   stencil.obj
 0001:00062850       OVGCreateGeometryBuffer    10063850 f   geombuffer.obj
 0001:000628b8       OVGDestroyGeometryBuffer   100638b8 f   geombuffer.obj
 0001:00062904       OVGGetGeometryBufferAddresses 10063904 f   geombuffer.obj
 0001:00062a1c       OVGCheckStrideGranularityForTQ 10063a1c f   transfer.obj
 0001:00063854       OVGGenerateMipMaps         10064854 f   transfer.obj
 0001:000639e8       OVGCheckForMainTQFormat    100649e8 f   transfer.obj
 0001:00063a48       OVGCheckForValidTQImageSubDataFormat 10064a48 f   transfer.obj
 0001:00063af8       OVGTransferImageData       10064af8 f   transfer.obj
 0001:00063c44       OVGRemoveFont              10064c44 f   font.obj
 0001:00063d0c       vgCreateFont               10064d0c f   font.obj
 0001:00063de4       vgDestroyFont              10064de4 f   font.obj
 0001:00063e90       vgSetGlyphToPath           10064e90 f   font.obj
 0001:000640d8       vgSetGlyphToImage          100650d8 f   font.obj
 0001:000642a4       vgClearGlyph               100652a4 f   font.obj
 0001:00064450       vgDrawGlyph                10065450 f   font.obj
 0001:000647b8       vgDrawGlyphs               100657b8 f   font.obj
 0001:00064cb0       vgCreateEGLImageTargetKHR  10065cb0 f   eglimage.obj
 0001:00064e64       OVGGetImageSource          10065e64 f   eglimage.obj
 0001:00064ff4       PreToUnpre                 10065ff4 f   conversions.obj
 0001:00065170       UnpreToPre                 10066170 f   conversions.obj
 0001:000651dc       GreyLinearToNonLinear      100661dc f   conversions.obj
 0001:000652c0       RGBLinearToNonLinear       100662c0 f   conversions.obj
 0001:000653b0       RGBNonLinearToLinear       100663b0 f   conversions.obj
 0001:0006549c       GreyNonLinearToLinear      1006649c f   conversions.obj
 0001:00065578       RGBToGrey                  10066578 f   conversions.obj
 0001:00065624       AlphaSpace                 10066624 f   conversions.obj
 0001:0006563c       OnlyRedChannel             1006663c f   conversions.obj
 0001:00065650       ForceAlphaToOne            10066650 f   conversions.obj
 0001:00065660       ForceAlphaToMax            10066660 f   conversions.obj
 0001:00065670       QuantiseRedToTwoLevels     10066670 f   conversions.obj
 0001:000656b0       QuantiseAlphaToFourLevels  100666b0 f   conversions.obj
 0001:00065720       QuantiseOnlyAlphaToTwoLevels 10066720 f   conversions.obj
 0001:0006575c       ForceAlphaNotZeroToMax     1006675c f   conversions.obj
 0001:00065794       PrepareColourConversion    10066794 f   conversions.obj
 0001:000659d4       fl_Init                    100669d4 f   functionlist.obj
 0001:000659e4       fl_Add                     100669e4 f   functionlist.obj
 0001:00065a30       fl_Destroy                 10066a30 f   functionlist.obj
 0001:00065a68       OVG_GetTLSValue            10066a68 f   wince6_tls.obj
 0001:00065a98       OVG_SetTLSValue            10066a98 f   wince6_tls.obj
 0001:00065adc       PDSGeneratePixelEventProgram 10066adc f   pds.obj
 0001:00065c80       PDSGeneratePixelShaderSAProgram 10066c80 f   pds.obj
 0001:00065f28       PDSGeneratePixelShaderProgram 10066f28 f   pds.obj
 0001:00066178       PDSGenerateVertexShaderProgram 10067178 f   pds.obj
 0001:00066844       PDSGenerateTerminateStateProgram 10067844 f   pds.obj
 0001:000668ec       PDSPatchTerminateStateProgram 100678ec f   pds.obj
 0001:000668f8       WriteEndOfPassUSSECode     100678f8 f   pixevent.obj
 0001:00066910       WriteEndOfRenderUSSECode   10067910 f   pixevent.obj
 0001:00066940       WriteEndOfTileUSSECode     10067940 f   pixevent.obj
 0001:00066a00       UCH_CodeHeapCreate         10067a00 f   eurasiaconcmn:codeheap.obj
 0001:00066ad8       UCH_CodeHeapDestroy        10067ad8 f   eurasiaconcmn:codeheap.obj
 0001:00066c0c       UCH_CodeHeapFreeFunc       10067c0c f   eurasiaconcmn:codeheap.obj
 0001:00066c60       UCH_CodeHeapAllocateFunc   10067c60 f   eurasiaconcmn:codeheap.obj
 0001:00067150       CBUF_GetBufferSpace        10068150 f   eurasiaconcmn:buffers.obj
 0001:00067390       CBUF_UpdateBufferPos       10068390 f   eurasiaconcmn:buffers.obj
 0001:000673cc       CBUF_GetBufferDeviceAddress 100683cc f   eurasiaconcmn:buffers.obj
 0001:000673f0       CBUF_UpdateBufferCommittedPrimOffsets 100683f0 f   eurasiaconcmn:buffers.obj
 0001:00067478       CBUF_UpdateBufferCommittedHWOffsets 10068478 f   eurasiaconcmn:buffers.obj
 0001:000674bc       CBUF_UpdateTACtrlKickBase  100684bc f   eurasiaconcmn:buffers.obj
 0001:0006750c       CBUF_CreateBuffer          1006850c f   eurasiaconcmn:buffers.obj
 0001:0006764c       CBUF_DestroyBuffer         1006864c f   eurasiaconcmn:buffers.obj
 0001:00067668       FRM_Initialize             10068668 f   eurasiaconcmn:frameresource.obj
 0001:00067838       FRM_Attach                 10068838 f   eurasiaconcmn:frameresource.obj
 0001:00067944       FRM_IsResourceNeeded       10068944 f   eurasiaconcmn:frameresource.obj
 0001:00067aec       FRM_RemoveResourceFromAllLists 10068aec f   eurasiaconcmn:frameresource.obj
 0001:00067bc4       FRM_RemoveSurfaceReferences 10068bc4 f   eurasiaconcmn:frameresource.obj
 0001:00067c04       FRM_Destroy                10068c04 f   eurasiaconcmn:frameresource.obj
 0001:00067d6c       FRM_ReclaimUnneededResources 10068d6c f   eurasiaconcmn:frameresource.obj
 0001:00067d7c       FRM_DestroyUnneededGhosts  10068d7c f   eurasiaconcmn:frameresource.obj
 0001:00067d8c       PVRSRVCallocUserModeMem    10068d8c f   srvclum:SRVCLUM.dll
 0001:00067d9c       PVRSRVFreeUserModeMem      10068d9c f   srvclum:SRVCLUM.dll
 0001:00067dac       PVRSRVAllocUserModeMem     10068dac f   srvclum:SRVCLUM.dll
 0001:00067dbc       PVRSRVMemCopy              10068dbc f   srvclum:SRVCLUM.dll
 0001:00067dcc       PVRSRVUnlockMutex          10068dcc f   srvclum:SRVCLUM.dll
 0001:00067ddc       PVRSRVLockMutex            10068ddc f   srvclum:SRVCLUM.dll
 0001:00067dec       PVRSRVAllocDeviceMem       10068dec f   srvclum:SRVCLUM.dll
 0001:00067dfc       PVRSRVCreateMutex          10068dfc f   srvclum:SRVCLUM.dll
 0001:00067e0c       PVRSRVDestroyMutex         10068e0c f   srvclum:SRVCLUM.dll
 0001:00067e1c       PVRSRVFreeDeviceMem        10068e1c f   srvclum:SRVCLUM.dll
 0001:00067e2c       PVRSRVReallocUserModeMem   10068e2c f   srvclum:SRVCLUM.dll
 0001:00067e3c       PVRSRVMemSet               10068e3c f   srvclum:SRVCLUM.dll
 0001:00067e4c       PVRSRVPollForValue         10068e4c f   srvclum:SRVCLUM.dll
 0001:00067e5c       PVRSRVEventObjectWait      10068e5c f   srvclum:SRVCLUM.dll
 0001:00067e6c       SGXKickTA                  10068e6c f   srvclum:SRVCLUM.dll
 0001:00067e7c       PVRSRVFreeAppHintState     10068e7c f   srvclum:SRVCLUM.dll
 0001:00067e8c       PVRSRVGetAppHint           10068e8c f   srvclum:SRVCLUM.dll
 0001:00067e9c       PVRSRVCreateAppHintState   10068e9c f   srvclum:SRVCLUM.dll
 0001:00067eac       SGXQueueTransfer           10068eac f   srvclum:SRVCLUM.dll
 0001:00067ebc       KEGLGetDrawableParameters  10068ebc f   libimgegl:libIMGEGL.dll
 0001:00067ecc       KEGLUnbindImage            10068ecc f   libimgegl:libIMGEGL.dll
 0001:00067edc       KEGLResizeRenderSurface    10068edc f   libimgegl:libIMGEGL.dll
 0001:00067eec       KEGLGetImageSource         10068eec f   libimgegl:libIMGEGL.dll
 0001:00067efc       KEGLBindImage              10068efc f   libimgegl:libIMGEGL.dll
 0001:00067f0c       TlsCall                    10068f0c f   coredll:COREDLL.dll
 0001:00067f1c       TlsGetValue                10068f1c f   coredll:COREDLL.dll
 0001:00067f2c       TlsSetValue                10068f2c f   coredll:COREDLL.dll
 0001:00067f3c       DllMain                    10068f3c f   corelib0:dllmain.obj
 0001:00068058       _DllMainCRTStartup         10069058 f   corelib0:pegdmain.obj
 0001:00068088       __GSHandlerCheckCommon     10069088 f   corelib0:gshandler.obj
 0001:000680c4       __GSHandlerCheck           100690c4 f   corelib0:gshandler.obj
 0001:000680e8       __security_init_cookie     100690e8 f   corelib0:seccinit.obj
 0001:00068144       __security_check_cookie    10069144 f   corelib0:armsecgs.obj
 0001:00068158       __gsfailure                10069158 f   corelib0:armsecgs.obj
 0001:00068264       _cexit                     10069264 f   corelib0:cexit.obj
 0001:00068280       _initterm                  10069280 f   corelib0:crt0dat.obj
 0001:000682b4       _cinit                     100692b4 f   corelib0:crt0dat.obj
 0001:000682e8       memcpy                     100692e8 f   corelib1:COREDLL.dll
 0001:000682f8       memmove                    100692f8 f   corelib1:COREDLL.dll
 0001:00068308       strcmp                     10069308 f   corelib1:COREDLL.dll
 0001:00068318       memset                     10069318 f   corelib1:COREDLL.dll
 0001:00068328       memcmp                     10069328 f   corelib1:COREDLL.dll
 0001:00068338       free                       10069338 f   corelib1:COREDLL.dll
 0001:00068348       malloc                     10069348 f   corelib1:COREDLL.dll
 0001:00068358       _XcptFilter                10069358 f   corelib1:COREDLL.dll
 0001:00068368       __C_specific_handler       10069368 f   corelib1:COREDLL.dll
 0001:00068378       __security_gen_cookie2     10069378 f   corelib1:COREDLL.dll
 0001:00068388       __report_gsfailure         10069388 f   corelib1:COREDLL.dll
 0001:00068398       DisableThreadLibraryCalls  10069398 f   coredll:COREDLL.dll
 0001:000683a8       TerminateProcess           100693a8 f   coredll:COREDLL.dll
 0001:000683dc       __IMPORT_DESCRIPTOR_SRVCLUM 100693dc     srvclum:SRVCLUM.dll
 0001:000683f0       __IMPORT_DESCRIPTOR_libIMGEGL 100693f0     libimgegl:libIMGEGL.dll
 0001:00068404       __IMPORT_DESCRIPTOR_COREDLL 10069404     coredll:COREDLL.dll
 0001:00068418       __NULL_IMPORT_DESCRIPTOR   10069418     srvclum:SRVCLUM.dll
 0002:00000000       __imp_cos                  1006a000     corelib1:COREDLL.dll
 0002:00000004       __imp_DisableThreadLibraryCalls 1006a004     coredll:COREDLL.dll
 0002:00000008       __imp___report_gsfailure   1006a008     corelib1:COREDLL.dll
 0002:0000000c       __imp___security_gen_cookie2 1006a00c     corelib1:COREDLL.dll
 0002:00000010       __imp___C_specific_handler 1006a010     corelib1:COREDLL.dll
 0002:00000014       __imp__XcptFilter          1006a014     corelib1:COREDLL.dll
 0002:00000018       __imp___ged                1006a018     corelib1:COREDLL.dll
 0002:0000001c       __imp_exp                  1006a01c     corelib1:COREDLL.dll
 0002:00000020       __imp___itod               1006a020     corelib1:COREDLL.dll
 0002:00000024       __imp___utod               1006a024     corelib1:COREDLL.dll
 0002:00000028       __imp___dtou               1006a028     corelib1:COREDLL.dll
 0002:0000002c       __imp_sqrt                 1006a02c     corelib1:COREDLL.dll
 0002:00000030       __imp_malloc               1006a030     corelib1:COREDLL.dll
 0002:00000034       __imp_free                 1006a034     corelib1:COREDLL.dll
 0002:00000038       __imp___subd               1006a038     corelib1:COREDLL.dll
 0002:0000003c       __imp___addd               1006a03c     corelib1:COREDLL.dll
 0002:00000040       __imp_ceilf                1006a040     corelib1:COREDLL.dll
 0002:00000044       __imp_floorf               1006a044     corelib1:COREDLL.dll
 0002:00000048       __imp_pow                  1006a048     corelib1:COREDLL.dll
 0002:0000004c       __imp___rt_sdiv            1006a04c     corelib1:COREDLL.dll
 0002:00000050       __imp_memcmp               1006a050     corelib1:COREDLL.dll
 0002:00000054       __imp___dtoi               1006a054     corelib1:COREDLL.dll
 0002:00000058       __imp_TlsCall              1006a058     coredll:COREDLL.dll
 0002:0000005c       __imp_TlsGetValue          1006a05c     coredll:COREDLL.dll
 0002:00000060       __imp_TlsSetValue          1006a060     coredll:COREDLL.dll
 0002:00000064       __imp_memcpy               1006a064     corelib1:COREDLL.dll
 0002:00000068       __imp___utos               1006a068     corelib1:COREDLL.dll
 0002:0000006c       __imp___muls               1006a06c     corelib1:COREDLL.dll
 0002:00000070       __imp___adds               1006a070     corelib1:COREDLL.dll
 0002:00000074       __imp_sqrtf                1006a074     corelib1:COREDLL.dll
 0002:00000078       __imp___gts                1006a078     corelib1:COREDLL.dll
 0002:0000007c       __imp___divs               1006a07c     corelib1:COREDLL.dll
 0002:00000080       __imp___subs               1006a080     corelib1:COREDLL.dll
 0002:00000084       __imp___negs               1006a084     corelib1:COREDLL.dll
 0002:00000088       __imp___eqs                1006a088     corelib1:COREDLL.dll
 0002:0000008c       __imp___nes                1006a08c     corelib1:COREDLL.dll
 0002:00000090       __imp___lts                1006a090     corelib1:COREDLL.dll
 0002:00000094       __imp___les                1006a094     corelib1:COREDLL.dll
 0002:00000098       __imp___rt_udiv            1006a098     corelib1:COREDLL.dll
 0002:0000009c       __imp_fabsf                1006a09c     corelib1:COREDLL.dll
 0002:000000a0       __imp_TerminateProcess     1006a0a0     coredll:COREDLL.dll
 0002:000000a4       __imp_sin                  1006a0a4     corelib1:COREDLL.dll
 0002:000000a8       __imp___stod               1006a0a8     corelib1:COREDLL.dll
 0002:000000ac       __imp_acos                 1006a0ac     corelib1:COREDLL.dll
 0002:000000b0       __imp___dtos               1006a0b0     corelib1:COREDLL.dll
 0002:000000b4       __imp_fmodf                1006a0b4     corelib1:COREDLL.dll
 0002:000000b8       __imp___divd               1006a0b8     corelib1:COREDLL.dll
 0002:000000bc       __imp___muld               1006a0bc     corelib1:COREDLL.dll
 0002:000000c0       __imp___stou               1006a0c0     corelib1:COREDLL.dll
 0002:000000c4       __imp___ges                1006a0c4     corelib1:COREDLL.dll
 0002:000000c8       __imp_memmove              1006a0c8     corelib1:COREDLL.dll
 0002:000000cc       __imp_strcmp               1006a0cc     corelib1:COREDLL.dll
 0002:000000d0       __imp___itos               1006a0d0     corelib1:COREDLL.dll
 0002:000000d4       __imp___stoi               1006a0d4     corelib1:COREDLL.dll
 0002:000000d8       __imp_memset               1006a0d8     corelib1:COREDLL.dll
 0002:000000dc       __imp_atan                 1006a0dc     corelib1:COREDLL.dll
 0002:000000e0       __imp_floor                1006a0e0     corelib1:COREDLL.dll
 0002:000000e4       __imp___gtd                1006a0e4     corelib1:COREDLL.dll
 0002:000000e8       __imp___ltd                1006a0e8     corelib1:COREDLL.dll
 0002:000000ec       \177COREDLL_NULL_THUNK_DATA 1006a0ec     coredll:COREDLL.dll
 0002:000000f0       __imp_PVRSRVPollForValue   1006a0f0     srvclum:SRVCLUM.dll
 0002:000000f4       __imp_PVRSRVFreeUserModeMem 1006a0f4     srvclum:SRVCLUM.dll
 0002:000000f8       __imp_PVRSRVAllocUserModeMem 1006a0f8     srvclum:SRVCLUM.dll
 0002:000000fc       __imp_PVRSRVMemCopy        1006a0fc     srvclum:SRVCLUM.dll
 0002:00000100       __imp_PVRSRVUnlockMutex    1006a100     srvclum:SRVCLUM.dll
 0002:00000104       __imp_PVRSRVLockMutex      1006a104     srvclum:SRVCLUM.dll
 0002:00000108       __imp_SGXQueueTransfer     1006a108     srvclum:SRVCLUM.dll
 0002:0000010c       __imp_PVRSRVCreateAppHintState 1006a10c     srvclum:SRVCLUM.dll
 0002:00000110       __imp_PVRSRVGetAppHint     1006a110     srvclum:SRVCLUM.dll
 0002:00000114       __imp_PVRSRVFreeAppHintState 1006a114     srvclum:SRVCLUM.dll
 0002:00000118       __imp_SGXKickTA            1006a118     srvclum:SRVCLUM.dll
 0002:0000011c       __imp_PVRSRVEventObjectWait 1006a11c     srvclum:SRVCLUM.dll
 0002:00000120       __imp_PVRSRVCallocUserModeMem 1006a120     srvclum:SRVCLUM.dll
 0002:00000124       __imp_PVRSRVMemSet         1006a124     srvclum:SRVCLUM.dll
 0002:00000128       __imp_PVRSRVReallocUserModeMem 1006a128     srvclum:SRVCLUM.dll
 0002:0000012c       __imp_PVRSRVFreeDeviceMem  1006a12c     srvclum:SRVCLUM.dll
 0002:00000130       __imp_PVRSRVDestroyMutex   1006a130     srvclum:SRVCLUM.dll
 0002:00000134       __imp_PVRSRVCreateMutex    1006a134     srvclum:SRVCLUM.dll
 0002:00000138       __imp_PVRSRVAllocDeviceMem 1006a138     srvclum:SRVCLUM.dll
 0002:0000013c       \177SRVCLUM_NULL_THUNK_DATA 1006a13c     srvclum:SRVCLUM.dll
 0002:00000140       __imp_KEGLUnbindImage      1006a140     libimgegl:libIMGEGL.dll
 0002:00000144       __imp_KEGLResizeRenderSurface 1006a144     libimgegl:libIMGEGL.dll
 0002:00000148       __imp_KEGLGetImageSource   1006a148     libimgegl:libIMGEGL.dll
 0002:0000014c       __imp_KEGLBindImage        1006a14c     libimgegl:libIMGEGL.dll
 0002:00000150       __imp_KEGLGetDrawableParameters 1006a150     libimgegl:libIMGEGL.dll
 0002:00000154       \177libIMGEGL_NULL_THUNK_DATA 1006a154     libimgegl:libIMGEGL.dll
 0002:0000015c       __security_cookie          1006a15c     corelib0:seccinit.obj
 0002:00000160       __security_cookie_complement 1006a160     corelib0:seccinit.obj
 0002:00000168       _exitflag                  1006a168     corelib0:cexit.obj
 0002:0000016c       __onexitend                1006a16c     <common>
 0002:00000170       __onexitbegin              1006a170     <common>
 0002:00000174       _pRawDllMain               1006a174     <common>

 entry point at        0001:00068058

 Static symbols

 0001:0001c7c0       _InitialiseConversionTableNonLinearToLinear 1001d7c0 f   eglglue.obj
 0001:0001cea8       _InitialiseConversionTableLinearToNonLinear 1001dea8 f   eglglue.obj
 0001:0001d58c       _InitContext               1001e58c f   eglglue.obj
 0001:0001d7b4       _CreateShareableContextData 1001e7b4 f   eglglue.obj
 0001:0001e018       _DeleteShareableContextData 1001f018 f   eglglue.obj
 0001:0001e9dc       _ValidateImageFormatAsRenderFormat 1001f9dc f   eglglue.obj
 0001:0001efac       OVGNormaliseVector         1001ffac f   splines.obj
 0001:0001f098       OVGLineDistance            10020098 f   splines.obj
 0001:000210b8       OVGNormaliseVector         100220b8 f   ellipse.obj
 0001:00023928       OVGNormaliseVector         10024928 f   tessellate.obj
 0001:00023a14       OVGComputeNormal           10024a14 f   tessellate.obj
 0001:00023b5c       _PathUserToSurfaceMatrixChange 10024b5c f   tessellate.obj
 0001:00023c38       _StrokeLine                10024c38 f   tessellate.obj
 0001:00023de0       _StrokePoint               10024de0 f   tessellate.obj
 0001:00023f0c       _GenerateJoin              10024f0c f   tessellate.obj
 0001:00024988       _GenerateCap               10025988 f   tessellate.obj
 0001:000250f0       _IsShortStroke             100260f0 f   tessellate.obj
 0001:0002c6f4       OVGGetProcAddress          1002d6f4 f   get.obj
 0001:00030d04       _SetupUSSEVertexCodeForDepthClear 10031d04 f   clear.obj
 0001:00030dd8       _SetupUSSEVertexCodeForClear 10031dd8 f   clear.obj
 0001:000310cc       _SetupPixelShaderForClear  100320cc f   clear.obj
 0001:000356a0       _SetFRMError               100366a0 f   meminstance.obj
 0001:000356b8       _FreeMemInstanceFRM        100366b8 f   meminstance.obj
 0001:0003575c       _DestroyMemInstanceFRM     1003675c f   meminstance.obj
 0001:00036890       _SetPaintFormatTokens      10037890 f   paint.obj
 0001:0003696c       _OVGCalculateStops         1003796c f   paint.obj
 0001:00036b54       _ValidatePatternImage      10037b54 f   paint.obj
 0001:00039350       _InitRegs                  1003a350 f   sgxif.obj
 0001:000394f4       _StartFrame                1003a4f4 f   sgxif.obj
 0001:000395dc       _OVGOutputTerminateState   1003a5dc f   sgxif.obj
 0001:0003b6a4       _SetImageFormatTokens      1003c6a4 f   state.obj
 0001:0003c464       _SetupVertexShaderForAccum 1003d464 f   specobj.obj
 0001:0003cb04       OVGNormaliseVector         1003db04 f   pathutils.obj
 0001:0003f438       _GetMTEStateBlock          10040438 f   hwstate.obj
 0001:0003f880       _GenerateUSEMTEStateCopyCode 10040880 f   hwstate.obj
 0001:0003f9bc       _PatchMTEStateCopy         100409bc f   hwstate.obj
 0001:0003fce4       AddTileFillSection         10040ce4 f   pixelshader.obj
 0001:0003fe18       AddSwizzleSection          10040e18 f   pixelshader.obj
 0001:0003fecc       AddUnPremultiplySection    10040ecc f   pixelshader.obj
 0001:0003ff64       AddPremultiplySection      10040f64 f   pixelshader.obj
 0001:00040004       AddFakePreUnPreSection     10041004 f   pixelshader.obj
 0001:000400a0       AddNonLinearConversionSection 100410a0 f   pixelshader.obj
 0001:00040138       AddLinearConversionSection 10041138 f   pixelshader.obj
 0001:000401d0       AddImageMultiplySection    100411d0 f   pixelshader.obj
 0001:00040330       AddBlendSection            10041330 f   pixelshader.obj
 0001:000405c0       AddColourXFormSection      100415c0 f   pixelshader.obj
 0001:00040690       _CreatePixelCodeBlockFromSections 10041690 f   pixelshader.obj
 0001:000407ac       _PickPhase0Sections        100417ac f   pixelshader.obj
 0001:0004088c       _PickPhase1Sections        1004188c f   pixelshader.obj
 0001:00040ae4       _PickPhase2Sections        10041ae4 f   pixelshader.obj
 0001:00040dac       _AssemblePixelShaderPhase0 10041dac f   pixelshader.obj
 0001:00040edc       _SetUpInitialOperandLocations 10041edc f   pixelshader.obj
 0001:000410cc       _SetUpIteratorsForPixelShader 100420cc f   pixelshader.obj
 0001:00041288       _SetUpTAGUnitsForPixelShader 10042288 f   pixelshader.obj
 0001:000414c4       _SetUpPixelShaderPDSPrimaryProgram 100424c4 f   pixelshader.obj
 0001:00041704       _SetUpPixelShaderPDSSecondaryProgram 10042704 f   pixelshader.obj
 0001:000420b8       _AssembleVertexShaderPhase2 100430b8 f   vertexshader.obj
 0001:0004225c       _AssembleVertexShaderPhase1 1004325c f   vertexshader.obj
 0001:00042550       _AssembleVertexShaderPhase0 10043550 f   vertexshader.obj
 0001:000427cc       _SetUpUSEControlForVertexShader 100437cc f   vertexshader.obj
 0001:000428fc       _SetUpImageVertexBuffer    100438fc f   vertexshader.obj
 0001:0004337c       _SetUpVertexShaderPDSPrimaryProgram 1004437c f   vertexshader.obj
 0001:00043564       _SetUpVertexShaderPDSSecondaryProgram 10044564 f   vertexshader.obj
 0001:00043dd0       OVGGetActivePaint          10044dd0 f   hwscene.obj
 0001:00043fb0       _DrawPathPrimitive         10044fb0 f   hwscene.obj
 0001:0004489c       _CalcRegionClip            1004589c f   scissor.obj
 0001:00044954       _SetupVerticesForDrawmask  10045954 f   scissor.obj
 0001:00044bdc       _SetupVerticesAndShaderForDrawmask 10045bdc f   scissor.obj
 0001:00044e58       _SendScissorRect           10045e58 f   scissor.obj
 0001:00046504       _Adjust_Parent_FirstChild_NextSibling_Pointers 10047504 f   image.obj
 0001:00046784       _AlignRectangleWithImage   10047784 f   image.obj
 0001:0004f9c8       _SetupPixelShaderForMaskOp 100509c8 f   mask.obj
 0001:00050614       _SetupVertexShaderForMaskOp 10051614 f   mask.obj
 0001:00050878       _SetupVertexBufferForMaskOp 10051878 f   mask.obj
 0001:00052330       LargeDisplacement          10053330 f   subdivide.obj
 0001:00052c94       MaxFabsInterval            10053c94 f   subdivide.obj
 0001:00052d38       MulIntervals               10053d38 f   subdivide.obj
 0001:00052e68       SquareInterval             10053e68 f   subdivide.obj
 0001:00052f30       HighCurvature              10053f30 f   subdivide.obj
 0001:000534d4       AdjustControlPointsAndRetryStroking 100544d4 f   subdivide.obj
 0001:00053a48       SubdivideAtArbitraryPoint  10054a48 f   subdivide.obj
 0001:00053fb8       SolveQuadratic             10054fb8 f   subdivide.obj
 0001:00054450       LookForCusp                10055450 f   subdivide.obj
 0001:0005487c       OutputCuspFullCircle       1005587c f   subdivide.obj
 0001:00055114       NotDegenerated             10056114 f   subdivide.obj
 0001:00056dbc       _IF_TileFill               10057dbc f   imagefilter.obj
 0001:00056e50       _IF_TilePad                10057e50 f   imagefilter.obj
 0001:00056ea4       _IF_TileRepeat             10057ea4 f   imagefilter.obj
 0001:00056f5c       _IF_TileReflect            10057f5c f   imagefilter.obj
 0001:0005703c       _IF_OffsetStride           1005803c f   imagefilter.obj
 0001:00057060       _IF_OffsetTwiddle          10058060 f   imagefilter.obj
 0001:000570dc       _IF_ReadSrc32              100580dc f   imagefilter.obj
 0001:000571e0       _IF_ReadSrc16              100581e0 f   imagefilter.obj
 0001:000572e4       _IF_ReadSrc8               100582e4 f   imagefilter.obj
 0001:000573e8       _IF_ReadSrcOthers          100583e8 f   imagefilter.obj
 0001:00057554       _IF_ReadDst32              10058554 f   imagefilter.obj
 0001:00057658       _IF_ReadDst16              10058658 f   imagefilter.obj
 0001:0005775c       _IF_ReadDst8               1005875c f   imagefilter.obj
 0001:00057860       _IF_ReadDstOthers          10058860 f   imagefilter.obj
 0001:000579cc       _IF_Write32                100589cc f   imagefilter.obj
 0001:00057bd0       _IF_Write16                10058bd0 f   imagefilter.obj
 0001:00057dd4       _IF_Write8                 10058dd4 f   imagefilter.obj
 0001:00057fd8       _IF_WriteOthers            10058fd8 f   imagefilter.obj
 0001:00058254       _IF_Convert                10059254 f   imagefilter.obj
 0001:00058284       _IF_MaskingPre             10059284 f   imagefilter.obj
 0001:000584ec       _IF_MaskingNonpre          100594ec f   imagefilter.obj
 0001:00058530       _IF_PreparePreProc         10059530 f   imagefilter.obj
 0001:00058840       _IF_PreparePostProc        10059840 f   imagefilter.obj
 0001:00058b14       _PrepareConfig             10059b14 f   imagefilter.obj
 0001:00058bb8       _SeparableConvolve         10059bb8 f   imagefilter.obj
 0001:0005a2d8       __GaussianBlurThreeBoxes   1005b2d8 f   imagefilter.obj
 0001:0005c7bc       __GaussianBlurSkipSM       1005d7bc f   imagefilter.obj
 0001:0005f5b0       __GaussianBlurSeparableConvolve 100605b0 f   imagefilter.obj
 0001:00060d00       _MinAndMax                 10061d00 f   radialgradient.obj
 0001:00060dc0       _ClampGradientFocus        10061dc0 f   radialgradient.obj
 0001:00060f94       _CalculateRadialGradientUValue 10061f94 f   radialgradient.obj
 0001:00061468       _CalculateGradientGeometryRadiusScale 10062468 f   radialgradient.obj
 0001:00061590       _GenerateCachedUnitCircleVertices 10062590 f   radialgradient.obj
 0001:00061698       _GenerateCachedGradientGeometry 10062698 f   radialgradient.obj
 0001:00061898       _CheckRadialGradientParameters 10062898 f   radialgradient.obj
 0001:000619d8       _CompareMatrix             100629d8 f   radialgradient.obj
 0001:00061f58       _SetUpStencilVertexShaderPDSSecondaryProgram 10062f58 f   stencil.obj
 0001:00062408       _SetUpStencilVertexShaderPDSPrimaryProgram 10063408 f   stencil.obj
 0001:000624d4       _AssembleStencilVertexShaderUSECode 100634d4 f   stencil.obj
 0001:00062b10       OVGTransferColourToDevice  10063b10 f   transfer.obj
 0001:00062c2c       OVGTransferSystemToDevice  10063c2c f   transfer.obj
 0001:00062d94       OVGTransferNormalBlit      10063d94 f   transfer.obj
 0001:00062f94       OVGTransferNormalBlitScissoring 10063f94 f   transfer.obj
 0001:00063564       OVGTransferCustomBlit      10064564 f   transfer.obj
 0001:00065b7c       PDSEncodeSimpleMOVS        10066b7c f   pds.obj
 0001:00065bf8       PDSGetNextConstant         10066bf8 f   pds.obj
 0001:00065c3c       PDSGetNumConstants         10066c3c f   pds.obj
 0001:00066b44       CodeHeapInsertBlockInFreeList 10067b44 f   eurasiaconcmn:codeheap.obj
 0001:00066f80       GetBufferSpaceLeftInBytes  10067f80 f   eurasiaconcmn:buffers.obj
 0001:00066fe8       CheckUSSEBufferSpace       10067fe8 f   eurasiaconcmn:buffers.obj
 0001:000670bc       CheckTACtrlBufferSpace     100680bc f   eurasiaconcmn:buffers.obj
 0001:00067780       AllocAttachment            10068780 f   eurasiaconcmn:frameresource.obj
 0001:000679a4       WaitUntilResourceIsNotNeeded 100689a4 f   eurasiaconcmn:frameresource.obj
 0001:00067a30       RemoveResourceFromAllLists 10068a30 f   eurasiaconcmn:frameresource.obj
 0001:00067b18       RemoveSurfaceReferencesInList 10068b18 f   eurasiaconcmn:frameresource.obj
 0001:00067c78       ReclaimUnneededResourcesInList 10068c78 f   eurasiaconcmn:frameresource.obj
 0001:00067f5c       _DllMainCRTStartupHelper   10068f5c f   corelib0:pegdmain.obj
 0001:0006819c       doexit                     1006919c f   corelib0:cexit.obj
